:040000008A11D02968
:100090004D344934523449344E34443441340034BC
:1000A0000034003483120313A400240886008A114C
:1000B000DC208A110D30F100F10B5C2808007E086D
:1000C0008A007F0882005F208A118000840A040869
:1000D0007D0603190034FF0A0319FE0A6328831200
:1000E0000313A1000310003003180130A0003A30C0
:1000F000210203187C287D28862830302102031C29
:10010000822883288628A0010314A00D200C080053
:100110009828F930F0006400F00B8B288F286400D9
:10012000FF3083120313A4070318A50AFF30A507A5
:100130008312031325082404031D9F28A02889285F
:10014000080083120313A1000310003003180130CC
:10015000A000211CAC28AD28B1282208F0007008AE
:10016000A0070310A20D0310A10CA108031DB928BC
:10017000BA28A92820080800CE28250884002608C7
:100180008A1100228A118A1152208A1101308312A9
:100190000313A5070318A60A0030A607831203134A
:1001A0002508840026088A1100228A110038031DC0
:1001B000DA28DB28BD280800F91479088312031314
:1001C00085001030F000F00BE32864007915790801
:1001D0008312031385001030F000F00BED2864004B
:1001E000FB30F0007008F9057908831203138500CD
:1001F0001030F000F00BFA2864000800FD30F00029
:100200007008F90579088312031385001030F00097
:10021000F00B08296400791579088312031385000F
:100220001030F000F00B12296400FB30F000700871
:10023000F90579088312031385001030F000F00BE4
:100240001F29640008000310003003180130FB0070
:100250007B08B03E8400831300087606031D312915
:10026000322937297B08A03E84000008FA007B0869
:10027000013EFB0010307B02031C3F294029282946
:100280007A088312031386006430A4000030A500AE
:100290008A1188208A1108003034313432343334E2
:1002A00034343534363437343834393441344234E4
:1002B0004334443445344634EE34ED34EB34E734DF
:1002C000DE34DD34DB34D734BE34BD34BB34B73434
:1002D0007E347D347B347734503445345034533459
:1002E00049340034003400340034003400308312C8
:1002F0000313A0000030A100221C7F298029862939
:100300002408A0070318A10A2508A107013003103B
:10031000A40DA50DFF3E031D872901300310A30C7A
:10032000A20CFF3E031D8E2923082204031D9929D8
:100330009A297C292108A301A3072008A201A2076A
:100340000800F03083160313860083120313060897
:10035000C8004808F039F80076080F39F60076082A
:100360007804F6000608C8004808F039F800780854
:10037000F03A0319BC29BD29BE29B2290310003067
:10038000031801308316031386008A1123218A1172
:100390007A0883120313CA00C9010314C90D0800A7
:1003A000F601F701F801F901FA01FB01C701C801E3
:1003B000C901CA01CB0183160313CA01CB01CC01C9
:1003C000CD01CE01CF01D001D101D201831347303D
:1003D000FD000030FE004830FF003D3084008A11EF
:1003E00063208A11CA30FD000130FE004C30FF004E
:1003F000A03084008A1163208A1183018A11CA2DDA
:10040000FE00FE1F082A83137E18831700080800C9
:100410000408FE0002308A007E088207003401349E
:1004200000340A34003464340034E83403341034C3
:1004300027344434453450344F34533449345434DD
:10044000453400344F345034433449344F344E34FF
:100450003A3400344C344934533454344F34213416
:1004600000345234413434343D3430340034203498
:100470002434253432346434003452344134343436
:100480003D3431340034831203132B082A0403193A
:100490004A2A4B2A7B2AA7010314A70D5A2A0130A6
:1004A0000310AA0DAB0DFF3E031D502A0130F100D1
:1004B0007108A707AB1F5D2A5E2A4F2A2B08290265
:1004C000031D642A2A082802031C672A682A6E2A48
:1004D0002A08A8022B08031CA903A9020130031053
:1004E000AB0CAA0CFF3E031D6F2A0130A702031DAF
:1004F0007A2A7B2A5E2A2908A901A9072808A801C7
:10050000A807080083120313A600023086008A1190
:10051000FE208A110A3083120313A4000030A500C4
:100520008A1188208A11283083120313A20026081A
:100530008A11A1208A11F100831203132708710781
:10054000A6000310003003180130A700B62A1430AB
:1005500086008A11FE208A112130F100F10BAE2AAB
:100560000130F100710883120313A7072608270240
:10057000031CBB2ABC2AA72A0800013083120313DC
:1005800086008A11FE208A110A3083120313A40008
:0C0590000030A5008A1188208A110800A4
:1005A000003083120313A1000030A20026082504A6
:1005B0000319DB2ADC2A142BA0010314A00DEB2A5B
:1005C00001300310A50DA60DFF3E031DE12A0130E9
:1005D000F0007008A007A61FEE2AEF2AE02A0130DB
:1005E0000310A10DA20DFF3E031DF02A26082402D0
:1005F000031DFC2A25082302031CFF2A002B072BBE
:100600002508A3022608031CA403A4022114013018
:100610000310A60CA50CFF3E031D082B0130A00201
:10062000031D132B142BEF2A2208A401A407210871
:10063000A301A307080038308312031386008A1130
:10064000FE208A11053083120313A4000030A50098
:100650008A1188208A1138308312031386008A1188
:10066000FE208A112130F100F10B342B3830831237
:10067000031386008A11FE208A112130F100F10B4C
:100680003F2B38308312031386008A11FE208A1113
:100690002130F100F10B4A2B013083120313860045
:1006A0008A11FE208A11323083120313A400003015
:1006B000A5008A1188208A110D3083120313860049
:1006C0008A11FE208A112130F100F10B652B0630D2
:1006D0008312031386008A11FE208A112130F10053
:1006E000F10B702B08000310003003180130831247
:1006F0000313C9001830831603138500F0308600F9
:100700008113031000300318013083120313850096
:10071000EF30F600760886000430F700CD2B76081F
:10072000A800A9012808A4002908A5000230A600F5
:100730000030A7008A11D4238A1183138312031374
:100740002408F600760886000530A4000030A500D5
:100750008A1188208A1183120313061EB02BB12B35
:10076000BD2B861EB42BB52BBD2B061FB82BB92B6A
:10077000BD2B861BBC2BBD2BC02B8A11A1218A113E
:10078000831203134908013A031DC72BC82BCA2B38
:100790004A08D32B7708FF3EF700F708031DD12B3B
:1007A000D22B8F2B732B080003100030031801305D
:1007B00083120313A100A71FDE2BDF2BE72BA60953
:1007C000A709A60A0319A70AA1010314A10DA51FD1
:1007D000EA2BEB2BF42BA409A509A40A0319A50AFB
:1007E0000130F0007008A1060030A2000030A30024
:1007F000270826040319FD2BFE2B362CA001031419
:10080000A00D0D2C01300310A60DA70DFF3E031DFA
:10081000032C0130F0007008A007A71F102C112C2A
:10082000022C01300310A20DA30DFF3E031D122C5C
:1008300027082502031D1E2C26082402031C212C38
:10084000222C292C2608A4022708031CA503A50294
:10085000221401300310A70CA60CFF3E031D2A2C06
:100860000130A002031D352C362C112C2108031D4C
:100870003A2C3F2CA209A309A20A0319A30A2308B0
:10088000A501A5072208A401A407080083120313E9
:10089000B2003730AC00B22D3508253A0319512C7F
:1008A000522C5E2C3508F20032088400720883173F
:1008B00080000130F2007208B207B22D0030B300A0
:1008C0000030B4000310003003180130AE003608C9
:1008D0008A1109228A118A116F208A11031C712C36
:1008E000722CAF2C003083120313B3000030B4001D
:1008F0008312031336088A1109228A11F200F301C8
:100900003408A301A3073308A201A2070A30A400F8
:100910000030A5008A1176218A1172088313831290
:1009200003132207F40073080318730A2307F50062
:100930007408D03EB30075080318013EFF3EB400B2
:100940000130F2007208B60736088A1109228A11AE
:100950008A116F208A110318AE2CAF2C782C00015D
:10096000013883120313B6070001FF3836078A11D6
:1009700009228A11B500003A0319C12D643A0319FE
:10098000C52C0D3A0319C52CB22D2C0884008313F5
:100990000008AF00840A0008B0000230F2007208BC
:1009A000AC07B01FD42CD52CDE2C0330F20072081B
:1009B000AE04AF09B009AF0A0319B00AB5010314B8
:1009C000B50D3508F2007207013EF4008A110922C4
:1009D0008A11F300F40A74088A1109228A11F400BA
:1009E00074083002031DF62C73082F020318F92C2B
:1009F000FA2CFB2C052D0130F2007208B5073508E2
:100A0000053A031D042D052DE12C34083304031988
:100A10000A2D0B2D172D2E0803390319102D112D1A
:100A2000172DFF30B3070318B40AFF30B407350899
:100A3000F200F301F21BF3037308803AF400340868
:100A4000803A7402031D262D330872020318292DE3
:100A50002A2D382D831203133508F200F301F21BFF
:100A6000F3037208B3027308031CB403B4023E2DEF
:100A7000003083120313B3000030B4003408330491
:100A80000319432D442D5B2D2030F20032088400E1
:100A90007208831780000130F2007208B207FF303D
:100AA000B3070318B40AFF30B40734083304031D36
:100AB0005A2D5B2D442D2E0803390319602D612D0D
:100AC0006C2D2D30F20032088400720883178000EC
:100AD0000130F2007208B2073508AD00A82D3008C9
:100AE000A401A4072F08A301A3072D08F200720791
:100AF000013EF3008A1109228A11A500F30A730846
:100B00008A1109228A11A6008A11D0228A11831320
:100B1000831203132408A901A9072308A801A80721
:100B20000A30AA000030AB008A1143228A118313D5
:100B3000831203132808303EB5003508F20032084E
:100B400084007208831780000130F2007208B20737
:100B5000FF30F2007208AD072D08FF3A031DB12DDA
:100B6000B22D6F2D00010138B6070001FF3836079E
:100B70008A1109228A11B500B508031DC02DC12DA7
:100B80004C2C031032088400003003180130831706
:100B9000800008009A3084003D30B9000408BA0093
:100BA0000A30BB003908840083130008BC00B90A6E
:100BB0003A0884003C0883178000BA0ABB0BD22D88
:100BC00090308400C030B9000408BA000A30BB007D
:100BD0003908840083130008BC00B90A3A0884006D
:100BE0003C0883178000BA0ABB0BE82D9813073026
:100BF000831603139C0003100030031801309D007E
:100C000003100030031801309B000310003003185C
:100C100001308600183085008A111B238A118A1141
:100C2000BD228A1183120313051E172E182E1F2EA4
:100C30002F30A5000030A6008A11BC208A11831233
:100C40000313051A242E252E2C2E2330A500003048
:100C5000A6008A11BC208A118A1173238A118A1175
:100C6000BD228A11143083120313A5000030A600A0
:100C70008A11BC208A118A1173238A1183120313EB
:100C8000B900BA01390883160317AB0083120313A6
:100C90003A0883160317AC008A11BD228A11831605
:100CA00003172B088A1152208A11031000300318F1
:100CB000013083120313A70001308A1182228A11A6
:100CC0003030831603172B062C04031D682E692E63
:100CD000352F0A30AD000030AE009A308312031376
:100CE000A5008130A6008A11BC208A118A117323C5
:100CF0008A118A11BD228A119A3083120313A5002A
:100D00008130A6008A11BC208A110310003003181C
:100D1000013083120313A70001308A1182228A1145
:100D2000293083120313B6000A30B7000030B80030
:100D3000A4308A1146248A11A43083120313A5001B
:100D40008130A6008A11BC208A118A1173238A116E
:100D50008A11BD228A110B3083120313A5000030C3
:100D6000A6008A11BC208A1103100030031801303C
:100D700083120313A70001308A1182228A112930BD
:100D800083120313B6000A30B7000030B800A43055
:100D90008A1146248A11A43083120313A5008130DE
:100DA000A6008A11BC208A1183120313051ED92EB6
:100DB000DA2ED42E831603172D08FE3EAD002E0822
:100DC0000318013EFF3EAE002E082D04031DE92E40
:100DD000EA2E012F8A11BD228A111C3083120313BF
:100DE000A5000030A6008A11BC208A1183120313CB
:100DF0000514A030A4000F30A5008A1188208A11A4
:100E00000F2E031000300318013083120313A700C4
:100E100001308A1182228A11293083120313B6000D
:100E2000831603172E0883120313B801B80783161D
:100E300003172D0883120313B701B707A4308A11D3
:100E400046248A11A43083120313A5008130A60022
:100E50008A11BC208A11D03083120313A4000730FA
:100E6000A5008A1188208A11D42E31302B062C043B
:100E7000031D3B2F3C2F0F2E0830AF000030B00079
:100E8000903083120313A5008130A6008A11BC2084
:100E90008A118A1173238A118A11BD228A11903016
:100EA00083120313A5008130A6008A11BC208A1189
:100EB000031000300318013083120313A700013020
:100EC0008A1182228A11293083120313B600083056
:100ED000B7000030B800A4308A1146248A11A4302B
:100EE00083120313A5008130A6008A11BC208A1149
:100EF0008A1173238A118A11BD228A110B30831241
:100F00000313A5000030A6008A11BC208A1103102B
:100F100000300318013083120313A70001308A1137
:100F200082228A11293083120313B6000830B700D9
:100F30000030B800A4308A1146248A11A4308312EC
:100F40000313A5008130A6008A11BC208A118312E8
:100F50000313051EAC2FAD2FA72F831603172F08E1
:100F6000FE3EAF0030080318013EFF3EB0003008DF
:100F70002F04031DBC2FBD2FCA2F8A11BD228A1139
:100F80001C3083120313A5000030A6008A11BC2078
:100F90008A11F62E03100030031801308312031358
:100FA000A70001308A1182228A112930831203138B
:100FB000B60083160317300883120313B801B8076D
:100FC000831603172F0883120313B701B707A43042
:100FD0008A1146248A11A43083120313A50081309C
:100FE000A6008A11BC208A11D03083120313A400FA
:100FF0000730A5008A1188208A11A72F8A1100289E
:00000001FF
